:020000040000FA
:100000003528A00018200914200886008716000053
:1000100000000000000087120800A100182021083D
:10002000860087160000000000000000871208000C
:1000300089148316FF30860083120910871600008A
:1000400000000000000087120608A500A51B1E285E
:10005000891083168601831208002830A200A301AC
:10006000A30B3028A20B30280800850186018701E8
:100070008801890183163F3085008601DF308700C3
:10008000FF308800890182309F00831209153830C3
:100090000D202D2038300D202D2038300D202D2022
:1000A00001300D200C300D2080300D204530012016
:1000B0004E300120543001205230012041300120C7
:1000C00044300120413001205330012020300120F4
:1000D0004A30012032300120363001202D300120FD
:1000E0004A3001203330012037300120C0300D204C
:1000F0008316FF308600831209110508A600060842
:10010000A7000708A8000808A9000915AA20A72029
:10011000A420A1209E209B20982095202030012003
:10012000AD20B020B320B6207628A71FBC28B92860
:10013000271FBC28B928A71EBC28B928271EBC2801
:10014000B928A71DBC28B928271DBC28B928A71C79
:10015000BC28B928271CBC28B928291FBC28B928C5
:10016000A91FBC28B928261EBC28B928281CBC28D1
:0E017000B9283030012008003130012008008D
:02400E003A3F37
:00000001FF
